:0200000480007A
:100000009710000093800000171100001301810277
:1000100083A1000013020000930210001303F0FFFD
:10002000B70300809383F3FF3704008033F241006D
:10003000B3F2510033F36100B3F3710033F4810084
:100040002320310023224100232451002326610074
:1000500023287100232A8100971000009380C0FAA2
:1000600017110000130181FE03A400009304000097
:10007000130510009305F0FF370600801306F6FF06
:10008000B7060080B37494003375A400B375B40050
:100090003376C400B376D40023208100232291005C
:1000A0002324A1002326B1002328C100232AD10044
:1000B00097100000938080F517110000130181FA5A
:1000C00083A6000013070000930710001308F0FF39
:1000D000B70800809388F8FF3709008033F7E600FF
:1000E000B3F7F60033F80601B3F8160133F9260129
:1000F0002320D1002322E1002324F1002326010143
:1001000023281101232A210197100000938040F039
:1001100017110000130181F603A9000093090000E4
:10012000130A1000930AF0FF370B0080130BFBFF3C
:10013000B70B0080B3793901337A4901B37A590199
:10014000337B6901B37B7901232021012322310113
:10015000232441012326510123286101232A71010F
:1001600097100000938000EB17110000130181F23B
:1001700083AB0000130C0000930C1000130DF0FF74
:10018000B70D0080938DFDFF370E008033FC8B018F
:10019000B3FC9B0133FDAB01B3FDBB0133FECB01CF
:1001A0002320710123228101232491012326A1010F
:1001B0002328B101232AC101971C0000938CCCE5B0
:1001C000171D0000130D8DEE03AE0C001302F00797
:1001D0009302F0031303F0019303F0001304700083
:1001E00093043000B37E4E0033FF5E00B37F6F0098
:1001F000B3F07F0033F18000B371910023204D00F4
:100200002322CD012324DD012326ED012328FD0136
:10021000232A1D00232C2D00232E3D0097100000C3
:100220009380C0DF17110000130141EA03AE000004
:10023000B79DFFF7938D8D813370BE0123200100A0
:10024000971000009380C0DD17110000130141E8F2
:1002500003AE0000B79DFFF7938D8D813370BE0113
:10026000B3720000232001002322510097100000E8
:10027000938040DB17110000130101E683A1000009
:100280009303F0FF33F27100B372720033F3530043
:1002900033777300B377770033F87700B3FC03014B
:1002A00033FD9301B37D7D00232041002322A10172
:1002B0002324B101171500001305C5D797150000B9
:1002C000938545E2370610F01306C6F26306B502C1
:1002D0008326C5002320D600832685002320D60050
:1002E000832645002320D600832605002320D60040
:1002F000130505016FF09FFD370510F0130505F29A
:0403000023200500B1
:101000000000000001000000FFFFFFFFFFFFFF7F67
:1010100000000080FFFFCDAB7856341298BADCFE9A
:10102000145892360000000000000000000000008C
:10103000FFFFFFFFFFFFFFFFFFFFFFFFFFFFFFFFC0
:10104000FFFFFFFFFFFFFFFFFFFFFFFFFFFFFFFFB0
:10105000FFFFFFFFFFFFFFFFFFFFFFFFFFFFFFFFA0
:10106000FFFFFFFFFFFFFFFFFFFFFFFFFFFFFFFF90
:10107000FFFFFFFFFFFFFFFFFFFFFFFFFFFFFFFF80
:10108000FFFFFFFFFFFFFFFFFFFFFFFFFFFFFFFF70
:10109000FFFFFFFFFFFFFFFFFFFFFFFFFFFFFFFF60
:1010A000FFFFFFFFFFFFFFFFFFFFFFFFFFFFFFFF50
:1010B000FFFFFFFFFFFFFFFFFFFFFFFFFFFFFFFF40
:1010C000FFFFFFFFFFFFFFFFFFFFFFFFFFFFFFFF30
:1010D000FFFFFFFFFFFFFFFFFFFFFFFFFFFFFFFF20
:040000058000000077
:00000001FF
